:100000000C949D000C94BA000C94BA000C94BA00A5
:100010000C94BA000C94BA000C94BA000C94BA0078
:100020000C94BA000C94BA000C94BA000C94B70269
:100030000C940F030C94BA000C94BA000C94BA0000
:100040000C94BA000C94BA000C94BA000C94BA0048
:100050000C94BA000C94BA000C94BA000C94BA0038
:100060000C94BA000C94BA000C94BA000C94BA0028
:100070000C94BA000C94BA000C94BA000C94BA0018
:100080000C94BA000C94BA000C94BA000C94BA0008
:100090000C94BA000C94BA0000010000C1001200D8
:1000A000020000D3001900030000EC000401030962
:1000B00004F00028020309041A011E000001C10611
:1000C000001201000200000020C0167C04000101A3
:1000D00002000109021900010100C03209040000F8
:1000E00001FF01010007058303080001040309045F
:1000F00028035B004D0061006E0075006600610022
:1001000063007400750072006500720020006800D2
:100110006500720065005D0000001E035B0050007A
:1001200072006F00640075006300740020006800B6
:100130006500720065005D00000011241FBECFEF56
:10014000D2E0DEBFCDBF11E0A0E0B1E0E4EAF0E133
:1001500002C005900D92AC38B107D9F711E0ACE8B8
:10016000B1E001C01D92A839B107E1F70E94610119
:100170000C9450080C9400008091E80080FFFCCFA4
:1001800008958091E80082FFFCCF08958EBD0DB4E4
:1001900007FEFDCF08958A3010F4805D01C0895CB0
:1001A0000E94C60008951F93182F82958F700E9499
:1001B000CB00812F8F700E94CB001F9108950E9469
:1001C000C6000895559A8AE08A95F1F700C0569ABC
:1001D000089598E02AE02A95F1F700C087FF02C051
:1001E000559801C0559A2AE02A95F1F700C0569813
:1001F00025E12A95F1F70000569A915011F0880FE9
:10020000E9CF559885E18A95F1F70000569825E1E8
:100210002A95F1F7000099B1569A8AE08A95F1F78C
:1002200000C081E095FF80E008959C01559898E01A
:1002300080E04AE04A95F1F700C0569845E14A95BA
:10024000F1F70000880F4D9981604AE04A95F1F777
:1002500000C0569A915069F72115310509F4559A55
:100260009AE09A95F1F700C0569840E24A95F1F766
:10027000569A9AE09A95F1F700C0559808955698C5
:100280008AE08A95F1F700C0559808951F93DF938F
:10029000CF930F92CDB7DEB7182F69830E94E2008B
:1002A0008CE30E94E900812F0E94E9006981862F7A
:1002B0000E94E9000E943F010F90CF91DF911F91B2
:1002C00008958F929F92AF92BF92CF92DF92EF925A
:1002D000FF920F931F93DF93CF930F92CDB7DEB7AB
:1002E000F89481E08AB9239A84B1887F84B980E444
:1002F0008CBD8CE791E0909395018093940180E808
:10030000809361001092610010928F0180EA8093C7
:10031000D8001092630086E089BD09B400FEFDCFCD
:1003200080E88093D8001092E0008CE08093E20097
:100330007894FF2403C00E94C600F394EF2DF0E0F0
:10034000E050FF4F80818823B1F78BB18F798BB953
:100350008AB18F798AB98FEF91EEA4E081509040F5
:10036000A040E1F700C000000E94E20082E30E948A
:10037000E900882381F0FF2403C00E94C600F394A3
:10038000EF2DF0E0E95FFE4F80818823B1F70E94F6
:100390003F0191E032C080E20E94E90087E70E94BD
:1003A000E9000E943F019AE09A95F1F700C00E948F
:1003B000E2008CE30E94E900882381F0FF2403C05F
:1003C0000E94C600F394EF2DF0E0EE5EFE4F8081B8
:1003D0008823B1F70E943F0192E00FC080E00E94A5
:1003E000E9008CE90E94E90080E20E94E90080E0D7
:1003F0000E94E9000E943F0190E080E060E899835C
:100400000E94460181E060EE0E9446019981892F99
:100410000E94D3000E94E20082E30E94E90088EA81
:100420000E94E9000E943F01AAE0AA95F1F700C0EE
:100430000E94E20083E30E94E90080E090E00E94D5
:10044000150180E090E00E94150180E090E00E949C
:10045000150180E090E00E94150180E090E00E948C
:10046000150181E090E00E9415010E943F01BAE071
:10047000BA95F1F700C00E94E2008CE30E94E90007
:1004800083E80E94E9000E943F01EAE0EA95F1F763
:1004900000C00E94E2008DE30E94E90080E090E04D
:1004A0000E941501D82E80E090E00E941501C82E10
:1004B00080E090E00E94150180E090E00E9415012C
:1004C00080E090E00E941501F82E81E090E00E940B
:1004D0001501E82E0E943F01FAE0FA95F1F700C0FD
:1004E0000E94E2008CE30E94E90081EB0E94E90097
:1004F0000E943F018AE08A95F1F700C00E94E20065
:100500008DE30E94E90080E090E00E94150181E007
:1005100090E00E9415010E943F0182E061E00E948C
:10052000460180E00E94C60080E20E94C6009D2C29
:100530008824DD24C828D9288D2D0E94D3008C2D35
:100540000E94D30080E20E94C6001F2D00E0FF241D
:10055000E02AF12A8F2D0E94D3008E2D0E94D30015
:1005600080E20E94C6008AE00E94C60053CF1F921C
:100570000F920FB60F9211248F939F938091E100F9
:100580001092E10083FF0FC01092E90091E0909378
:10059000EB001092EC0092E29093ED0098E09093C3
:1005A000F0001092900182FF33C080919001882367
:1005B00079F180918D0190918E01009749F1019719
:1005C00090938E0180938D0183E08093E900809168
:1005D000E80085FF1DC01092F10081ED8093F100CD
:1005E00082ED8093F10083ED8093F10084ED8093A0
:1005F000F10085ED8093F10086ED8093F10087EDA9
:100600008093F10088ED8093F1008AE38093E80005
:100610009F918F910F900FBE0F901F9018951F9272
:100620000F920FB60F921124AF92BF92DF92EF920A
:10063000FF920F931F932F933F934F935F936F936B
:100640007F938F939F93AF93BF93EF93FF93DF932A
:10065000CF930F92CDB7DEB71092E9000091E8007A
:100660008AE290E00E944D0503FFE4C1D090F100C2
:100670002091F1008091F100A82EBB243091F1006F
:10068000932F80E0A82AB92A0091F10010E0309160
:10069000F100932F80E0082B192BE090F100FF244C
:1006A0003091F100932F80E0E82AF92A8DB79EB7A8
:1006B0000C970FB6F8949EBF0FBE8DBFEDB7FEB777
:1006C00031968DE191E0ADB7BEB712969C938E93B3
:1006D0001197D282138224831582B782A682118752
:1006E0000087F386E28629830E94380582EF809393
:1006F000E800EDB7FEB73C960FB6F894FEBF0FBE0C
:10070000EDBF2981263009F054C08FE990E09C01AB
:1007100025503040FC013797459154914A155B05AF
:10072000D1F4F9014591549140175107A1F42E5F7E
:100730003F4FF901859194912E5F3F4FF90124912C
:10074000A7014F3F510519F010F04FEF50E042174D
:1007500050F4242F08C00796295F3F4FF0E0823CF9
:100760009F07C1F667C1AEEF4091E80050E0BA01C3
:100770006570707061157105B9F342FD5EC1322F6D
:10078000213208F030E2AC01632F07C0FA014F5F5D
:100790005F4FE491E093F10061506623B9F7830F56
:1007A000911D231BA093E8002223F1F63032E1F2E1
:1007B00044C1253051F48EEF8093E8000E94BC00C4
:1007C0008A2D80688093E30038C1293051F5DD20FF
:1007D00009F0CFC0A09290018EEF8093E80041E035
:1007E0008BEB90E04093E900FC010196E491E093EB
:1007F000EB00EE2369F09C012F5F3F4FFC018491D9
:100800008093EC00C9010196F90124912093ED0039
:100810004F5F453039F78EE18093EA001092EA008D
:100820000CC1283049F4FD2DF03809F0A2C00E9417
:10083000BC0080919001DDC0222399F40E94BC008D
:100840002D2D223851F40093E9009091EB0081E0C6
:1008500095FF80E01092E90001C080E08093F100F4
:10086000B8C0233AC9F48091E80090E0AC0145702B
:10087000507041155105B9F382FDDFC08BE08093C4
:10088000F1008150E1F78EEF8093E80080E491E081
:1008900029830E94540583C0243AF1F40E94BC00CD
:1008A00034E03093F10025E02093F10096E090933E
:1008B000F10087E08093F1003093F1002093F10084
:1008C0009093F1008093F1008EEF8093E8008DE427
:1008D00091E00E945405B1C0263AA9F488E591E060
:1008E0000E9454058091E80090E09C0125703070D2
:1008F00021153105B9F382FDA0C08FE18093F1008D
:100900008150E1F793C0253AA1F50E94C10000D0C3
:100910008CE591E0ADB7BEB712969C938E9311977C
:100920000E9438050F900F90AA24BB2408E611E01E
:1009300018C08091F10000D000D0EDB7FEB731961D
:10094000ADB7BEB712961C930E9311978283138294
:100950000E9438050894A11CB11C0F900F900F90B5
:100960000F90AE14BF0428F38AE090E00E944D057A
:100970004EC000D000D0EDB7FEB731968EE691E0C4
:10098000ADB7BEB712969C938E93119722831382B4
:1009900029830E9438050F900F900F900F902981A6
:1009A0000115110509F046C0BD2DB13A29F52130D8
:1009B00099F40E94BC001092F1001092F100109284
:1009C000F1001092F1001092F1001092F1001092DB
:1009D000F1001092F1002AC0223029F40E94BC00DC
:1009E00080918A0106C0233029F50E94BC008091C5
:1009F0008B018093F1001AC0ED2DE132D9F429303A
:100A000051F40E94C1008091F10080938C018BEF22
:100A10008093E8000BC02A3029F4B0928A0110922A
:100A2000910104C02B3031F4A0928B018EEF8093A2
:100A3000E80003C081E28093EB000F90CF91DF913B
:100A4000FF91EF91BF91AF919F918F917F916F91A6
:100A50005F914F913F912F911F910F91FF90EF90D8
:100A6000DF90BF90AF900F900FBE0F901F90189522
:100A7000A0E0B0E0EEE3F5E00C942908FE01359625
:100A8000619171918091940190919501AF010E94C3
:100A900089052096E2E00C944508609194017091DC
:100AA00095010E9484070895EF92FF920F931F9380
:100AB000CF93DF938C01E0919401F09195018381B4
:100AC00081FF1FC0C0E0D0E00AC0DB011896ED91A5
:100AD000FC9119970995009711F0CFEFDFEFF8011E
:100AE00081918F016091940170919501882369F73C
:100AF000DB011896ED91FC9119978AE00995009712
:100B000011F0CFEFDFEFCE01CDB7DEB7E6E00C940A
:100B10004108ACE0B0E0EFE8F5E00C9419086C0196
:100B20001B018A01FC0117821682838181FFCFC1DC
:100B30002E010894411C511CF6019381F10193FD93
:100B4000859193FF81911F01882309F4BCC18532EF
:100B500039F493FD859193FF81911F01853229F42A
:100B600090E0B6010E948407E7CFEE24FF2420E046
:100B70002032B0F48B3269F08C3228F4803251F09C
:100B8000833271F40BC08D3239F0803349F4216027
:100B90002AC02260246027C0286025C0206123C0AD
:100BA00027FD2AC0382F30533A3088F426FF07C07B
:100BB0008E2D6AE00E941008E82EE30E14C08F2DDF
:100BC0006AE00E941008F82EF30E20620CC08E32EC
:100BD00021F426FD78C1206406C08C3611F420680B
:100BE00002C0883649F4F10193FD859193FF81910C
:100BF0001F01882309F0BCCF982F9554933018F02B
:100C00009052933028F40C5F1F4FFFE3F9830DC01F
:100C1000833631F0833771F0833509F060C022C02C
:100C2000F801808189830E5F1F4F420171E0A72E7A
:100C3000B12C16C062E0662E712C600E711EF80198
:100C40008080918026FF03C06E2D70E002C06FEFA0
:100C50007FEFC4012C870E9479075C0183012C85FA
:100C60002F7717C052E0652E712C600E711EF801AF
:100C70008080918026FF03C06E2D70E002C06FEF70
:100C80007FEFC4012C870E946E075C012C852068D1
:100C9000830123FD20C008C080E290E0B6012C87CC
:100CA0000E948407FA942C858F2D90E0A816B9062F
:100CB00098F311C0F40127FD859127FF81914F0121
:100CC00090E0B6012C870E9484072C85F110FA94DD
:100CD0000894A108B108A114B10461F7F1C08436E9
:100CE00011F0893649F527FF08C0F801608171814C
:100CF000828193810C5F1F4F09C0F801608171816F
:100D0000882777FD8095982F0E5F1F4F4FE6B42EF2
:100D1000B22297FF09C090958095709561957F4F9D
:100D20008F4F9F4FF0E8BF2AA2012AE030E00E94D7
:100D3000B007782E741845C0853731F43FEEB32ED6
:100D4000B2222AE030E025C099EFB92EB2228F36C8
:100D5000C1F0803720F4883509F0B5C00DC0803768
:100D600021F0883709F0AFC002C020E1B22AB4FEFA
:100D70000BC084E0B82A08C0B4FE09C0E6E0BE2A71
:100D800006C028E030E005C020E130E002C020E1EC
:100D900032E0B7FE08C0F8016081718182819381E1
:100DA0000C5F1F4F07C0F8016081718180E090E007
:100DB0000E5F1F4FA2010E94B007782E7418FFE744
:100DC000BF22B6FE0BC02EEFB2227E1438F4B4FE62
:100DD00007C0B2FC05C08FEEB82202C0A72C01C02C
:100DE000AE2C8B2D90E0B4FE0DC0FE01E70DF11D81
:100DF0002081203319F4E9EEBE2209C0A394B2FE8B
:100E000006C004C086789070009709F0A3948B2CDC
:100E10009924B3FC14C0B0FE0FC0AF1428F4E72C23
:100E2000EF0CEA18AF2C08C0E72C06C080E290E077
:100E3000B6010E948407A394AF14C0F304C0AF149A
:100E400010F4FA1801C0FF2484FE0FC080E390E084
:100E5000B6010E94840782FE1FC081FE03C088E5A0
:100E600090E010C088E790E00DC0C40186789070D3
:100E7000009791F081FC02C080E201C08BE2B7FCD8
:100E80008DE290E0B6010E94840706C080E390E006
:100E9000B6010E948407EA947E14C0F37A94F201AA
:100EA000E70DF11D808190E0B6010E948407772054
:100EB000A9F706C080E290E0B6010E948407FA9488
:100EC000FF20C1F739CEF6012681378102C02FEF0E
:100ED0003FEFC9012C96E2E10C943508FC01059026
:100EE000615070400110D8F7809590958E0F9F1F2C
:100EF0000895FC016150704001900110D8F7809571
:100F000090958E0F9F1F08950F931F93CF93DF939C
:100F10008C01EB018B8181FF1BC082FF0DC02E81F4
:100F20003F818C819D812817390764F4E881F9811C
:100F30000193F983E88306C0E885F985802F099538
:100F4000009731F48E819F8101969F838E8302C02A
:100F50000FEF1FEFC801DF91CF911F910F910895FF
:100F6000FA01AA27283061F1203191F1E8946F93BA
:100F70006E7F6E5F7F4F8F4F9F4FAF4FB1E040D07E
:100F8000B4E03ED0670F781F891F9A1FA11D680F1C
:100F9000791F8A1F911DA11D6A0F711D811D911D51
:100FA000A11D22D009F468943F91062E000C30193F
:100FB000000C000C3019305D3193CEF6CF0108954E
:100FC000462F4770405D4193B3E00FD0C9F7F6CF8D
:100FD000462F4F70405D4A3318F0495D31FD405255
:100FE000419302D0A9F7EACFB4E0A69597958795EB
:100FF00077956795BA95C9F70097610571050895CA
:101000009B01AC010A2E0694579547953795279575
:10101000BA95C9F7620F731F841F951FA01D08950D
:10102000002480FD060E660F11F08695D1F7802D05
:1010300008952F923F924F925F926F927F928F927C
:101040009F92AF92BF92CF92DF92EF92FF920F9357
:101050001F93CF93DF93CDB7DEB7CA1BDB0B0FB661
:10106000F894DEBF0FBECDBF09942A88398848881E
:101070005F846E847D848C849B84AA84B984C884B4
:10108000DF80EE80FD800C811B81AA81B981CE0FAB
:10109000D11D0FB6F894DEBF0FBECDBFED01089590
:0410A000F894FFCFF2
:1010A40053746172740A004C494E204641494C2ED7
:1010B4000A004D4147204641494C2E0A00524551F1
:1010C4003A20253032782025303278202F202530E0
:1010D40034782C20253034782C20253034780A00BC
:1010E40030784133202F20646174613A00307841B4
:1010F4003420476F6F642E0041362E00307841351E
:101104002053656E643A2000202530325800554E35
:101114004B5245513A20253032580A000000000253
:0C11240000000000DF00000000007D0162
:00000001FF
